:020000021000EC
:10F00000CFEFD0E1DEBFCDBF87E089B988E18AB913
:10F010001124F89484EF9FEF9C01442737FD40951D
:10F02000542FA0E0B1E081E0A630B80760F44BBFF8
:10F03000F90187918D932F5F3F4F4F4F5F4F81E0D5
:10F04000A630B807A0F3A6E0B1E086E0AE36B80778
:10F0500028F41D9286E0AE36B807D8F30E94B0FDC2
:10F060000E9419FA892B31F480916403882311F0EE
:10F070000E9496F80C940000FFCFCF92DF92EF929F
:10F08000FF920F931F93CF93DF937C018A016B0153
:10F090004150514010F000E011E0EFEFEE16F104A6
:10F0A00049F040F0F0EEEF16F1E0FF06B0F581E038
:10F0B0008BBF01C01BBEFE2CEE2463E0C7010E9483
:10F0C000ECFF61E180E090E00E94ECFFC0E0D0E066
:10F0D000C017D10758F4F601619171916F01CE010B
:10F0E0000E94EEFF2296C017D107A8F3CF3FD105AB
:10F0F00009F050F46FEF7FEFCE010E94EEFF2296F1
:10F10000CF3FD105B9F3B0F365E0C7010E94ECFF32
:10F1100061E180E090E00E94ECFFDF91CF911F91D0
:10F120000F91FF90EF90DF90CF9008958F929F9274
:10F13000AF92BF92CF92DF92EF92FF920F931F9305
:10F14000CF93DF93EE24FF2455E4852E912C5701B5
:10F1500081E090E0082E892F902D909313048093E6
:10F16000120442E0C42ED12CE4E1F4E0A4E6B3E0C2
:10F170002D9121930894C11CD11C2223C9F78FE63D
:10F18000819383E6819394E7919385E681939193AC
:10F19000208386E090E0C80ED91EC0E080910A016D
:10F1A00090910B01A0910C01B0910D01860120E01E
:10F1B00034E0A401BC01CD010E941BFB97FD0BC0F4
:10F1C00068E873E180E094E00E94F7FA7C0194E043
:10F1D000E916F1041CF4CF5FC33000F384E0E816B5
:10F1E000F1040CF42EC08091380190913901082E61
:10F1F000892F902D039729F5A114B10499F48090DB
:10F20000300190903101082C892C902C84E090E002
:10F21000082E892F902D909313048093120434E0CC
:10F22000C32ED12C80913A0190913B01082E892F59
:10F23000902DE50121968C179D0731F0A114B104A2
:10F2400059F58FEF9FEF40C095E0E916F104DCF02F
:10F25000C70104978501000F111FAC016CE371E039
:10F26000C8010E943DF885E0E81681E0F8065CF0F0
:10F27000C701845091400F5F1F4FAC016CE372E0F7
:10F28000C8010E943DF85E01CE01082E892F902D05
:10F29000909315048093140494E0E91692E0F90623
:10F2A0000CF07BCF80910A0190910B01A0910C0191
:10F2B000B0910D01860120E034E0A401BC01CD0134
:10F2C0000E941BFB80E090E0DF91CF911F910F9196
:10F2D000FF90EF90DF90CF90BF90AF909F908F9076
:10F2E0000895CF93DF93982FC8E2D2E088818823D6
:10F2F000F1F08F3FF1F08917B1F48981841708F498
:10F30000482F90E0941760F4E92FFF27DB01AE0F40
:10F31000BF1FEC0FFD1F82818C939F5F9417A0F39A
:10F320008981992708C021968881C80FD11D21960F
:10F33000DDCF80E090E0DF91CF910895FC01DA010C
:10F340006193219321502F3F21F08D918193215082
:10F35000E0F78FEF8083CF010895CF92DF92EF9295
:10F36000FF920F931F93CF93DF93CDB7DEB7219713
:10F370000FB6F894DEBF0FBECDBF6C01E62EFF24A2
:10F38000860124E430E043E450E06FEF7FEF8FEF3D
:10F390009FEF0E941BFB99234CF068E873E184E423
:10F3A00090E00E94F7FA8C0197FF03C08FEF9FEF68
:10F3B00031C0892B09F120913C0130913D014091F0
:10F3C0003E0150913F018091160490911704A09145
:10F3D0001804B0911904281739074A075B0761F42C
:10F3E00041E0BE016F5F7F4F85E30E9471F981307C
:10F3F00019F489818E1569F000E010E068EE73E081
:10F4000080E090E00E94D9FFF39482E08F1508F02D
:10F41000B7CFC80121960FB6F894DEBF0FBECDBF9F
:10F42000DF91CF911F910F91FF90EF90DF90CF90E0
:10F4300008951F93CF93DF93CDB7DEB721970FB613
:10F44000F894DEBF0FBECDBF21E02093120481E00F
:10F4500092E0A3E0B4E08093160490931704A09385
:10F460001804B093190480E890E090931D048093F1
:10F470001C042093130486E080931404198290E006
:10F48000AEE2B4E0E0E0F1E081918D93892F8F5FEF
:10F49000982F8630C8F383E692E8A3E5B3E680931D
:10F4A000FE049093FF04A0930005B093010511E0C2
:10F4B0001983212FAE014F5F5F4F65E382E095E036
:10F4C0000E949EF962E084EF90E00E94ADF9181668
:10F4D00019062CF544E064EE73E086E30E9471F9AE
:10F4E00083E08983212FAE014F5F5F4F65E382E0A8
:10F4F00095E00E949EF924E048E451E062E30E9416
:10F500009EF924E044EE53E066E30E949EF965E034
:10F5100080E091E00E94ADF9181619061CF08FEFFB
:10F520009FEF5BC08091480190914901A0914A01F1
:10F53000B0914B018093060190930701A0930801BD
:10F54000B093090180914C0190914D01A0914E0121
:10F55000B0914F0180930A0190930B01A0930C018D
:10F56000B0930D010097A105B10581F480912801A8
:10F5700090912901A0912A01B0912B0180930A0159
:10F5800090930B01A0930C01B0930D01E4EAF1E01C
:10F5900019828091A401882361F09981A4E6B3E0E7
:10F5A00081918D939F5F99838081882311F09F378C
:10F5B000B8F38981E82FFF27EC59FC4F108244E013
:10F5C00060E673E081E00E9471F944E064EE73E06C
:10F5D00086E30E9471F980E090E021960FB6F894DE
:10F5E000DEBF0FBECDBFDF91CF911F9108950F9366
:10F5F0001F93CF93DF938C01EB01BE0181E10E9449
:10F6000079FB1816190694F4809132019091330118
:10F61000082E892F902D0817190779F7809134014A
:10F6200090913501082E892F902D0897DF91CF9169
:10F630001F910F910895CF92DF92EF92FF920F9357
:10F640001F936B017C01C9019801082E892F902D11
:10F6500090930B0480930A04042E452F502D509351
:10F660000D0440930C04C8010896082E892F902D94
:10F6700090930F0480930E04285F3F4F41E1C70130
:10F68000B6010E94E5FB1F910F91FF90EF90DF9074
:10F69000CF900895FC0120E030E040E050E062307F
:10F6A000710558F081919191AA27BB27280F391F26
:10F6B0004A1F5B1F62507040F2CF672B29F0808198
:10F6C000280F311D411D511DCA01AA27BB27BC01AE
:10F6D000892B59F0620F731F9B0144275527CA01DC
:10F6E000AA27BB27BC01892BA9F7C9018095909552
:10F6F00008951F93CF93DF93182FEB01BE0188E08D
:10F7000090E00E94D9FEBC01181619060CF058C0F2
:10F7100020911C01822F807F803481F7809122010B
:10F7200090912301082E892F902D9F73892B31F7FB
:10F7300080912501811711F760911E0170911F01C1
:10F74000062E672F702D2F70822F9927880F991FF3
:10F75000880F991F681B790B20912C0130912D0186
:10F7600040912E0150912F012F3F8FEF38078FEFDF
:10F7700048078FEF580721F180910601909107010A
:10F78000A0910801B09109010097A105B10509F404
:10F79000B5CF281739074A075B0791F080916003BE
:10F7A00090916103A0916203B0916303282B392BE0
:10F7B0004A2B5B2B2F5F3F4F4F4F5F4F09F09ECF80
:10F7C000CB01DF91CF911F910895BF92CF92DF922D
:10F7D000EF92FF920F931F93CF93DF93CDB7DEB7D6
:10F7E00026970FB6F894DEBF0FBECDBF7B018C010C
:10F7F000B42E6901AE014F5F5F4F0E9460FC9C0117
:10F80000892B19F08FEF9FEF4BC085E48093F603AF
:10F81000C6014496082E892F902D9093F90380936A
:10F82000F80380E48093FE03B092FF03E0920604A5
:10F83000F0920704009308041093090480910601D4
:10F8400090910701A0910801B091090180930204F1
:10F8500090930304A0930404B09305048091FA03E9
:10F860009091FB0301969093FB038093FA033093EE
:10F8700001042093000464E170E086EF93E00E94AD
:10F880004AFB909301048093000484E190E0C80E49
:10F89000D91EA60168E070E0CE0101960E9441FEEB
:10F8A00026960FB6F894DEBF0FBECDBFDF91CF9185
:10F8B0001F910F91FF90EF90DF90CF90BF90089530
:10F8C000AF92BF92DF92EF92FF920F931F93CF936D
:10F8D000DF937B018C015A01C8E4D6E08FEFE81674
:10F8E0008FEFF8068FEF08078FEF180741F490E0CD
:10F8F000FA018FEF81939F5F9630D8F3C1C080915A
:10F90000640690916506A0916606B09167068E1513
:10F910009F05A007B10709F49AC081E090E0082E86
:10F92000892F902D909349068093480688E090E0B7
:10F9300090934B0680934A0686E080934C0684E0C1
:10F9400080934D0681E090E0082E892F902D9093B2
:10F950004F0680934E0690E0DE011896E0E0F1E05D
:10F9600081918D939F5F9630D8F38091060190919D
:10F970000701A0910801B09109018E879F87A88B8C
:10F98000B98B90E0EAE5F6E08FEF81939F5F9630C8
:10F99000D8F3E88EF98E0A8F1B8FDD244CE150E0FE
:10F9A00068E076E080E090E00E9441FE99230CF44C
:10F9B0004EC068EE73E088E096E00E94D9FE18160B
:10F9C00019060CF03DC0CCE1D1E02091340130911A
:10F9D0003501409136015091370180910601909197
:10F9E0000701A0910801B0910901281739074A07BA
:10F9F0005B0721F58091220190912301082E892F28
:10FA0000902D0297D9F480912A0190912B01A09119
:10FA10002C01B0912D018093640690936506A0930C
:10FA20006606B093670690E0A8E6B6E0FE01389659
:10FA300081918D939F5F9630D8F309C080E090E06C
:10FA4000D394892B21F489E08D1508F0A7CF8091FC
:10FA5000640690916506A0916606B09167068E15C2
:10FA60009F05A007B10719F08FEF9FEF0BC090E043
:10FA7000F501A8E6B6E08D9181939F5F9630D8F3AB
:10FA800080E090E0DF91CF911F910F91FF90EF9078
:10FA9000DF90BF90AF90089520916006309161068D
:10FAA0004091620650916306809106019091070192
:10FAB000A0910801B0910901281739074A075B078F
:10FAC00019F580914E0690914F06082E892F902DA2
:10FAD0000297D1F48091560690915706A09158064E
:10FAE000B09159068093640690936506A0936606CC
:10FAF000B093670690E0A8E6B6E0E0E5F6E0819115
:10FB00008D939F5F9630D8F3089580EC85BB84BBBE
:10FB100064E170E080E090E00E94D9FF81EE809384
:10FB2000008380E48093018385B78F7785BF80E071
:10FB300090E09D9B05C0019639F09D99FCCF04C0D3
:10FB4000019611F09D9BFCCF892B89F785B78068C2
:10FB500085BF15BA14BA809100838132E1F7089508
:10FB6000FF920F931F9300EC05BF10911F8365E078
:10FB700070E080E090E00E94D9FF10931F8368EE50
:10FB800073E080E090E00E94D9FF0E9485FD109212
:10FB90000F838FEFF82EF092078381EE809300831E
:10FBA000009301831092068310E210930583109254
:10FBB000018368EC70E080E090E00E94D9FF21E2D0
:10FBC0002093008388E480930E8310920A8310921E
:10FBD0000B8310930C8382E080930D8380E48093E9
:10FBE00004838FE5809303839CE49093018380E6F4
:10FBF00080930283F092078381E680930083809153
:10FC000000018093018380910101809302838091A0
:10FC10000201809303838091030180930483809188
:10FC200004018093058380910501809306831092DF
:10FC300008831092098310920A8310920B8310920A
:10FC40000C8310920D8310920E8310920F83909369
:10FC500007832093008384E080930C83F0920783D2
:10FC600010920F8382E28093008310920D8368EEDE
:10FC700073E080E090E00E94D9FF1F910F91FF9008
:10FC80000895EF92FF920F931F93CF93DF938C0110
:10FC900086E06830780729F43AE3E32E36E0F32E65
:10FCA00004C028EEE22E23E0F22EE701D7011696DB
:10FCB000E0E0F1E09F012B5F3F4F81918D932E1784
:10FCC0003F07D8F70115110559F0FE01D8019E0133
:10FCD0002B5F3F4F8D9181932E173F07D8F709C0B7
:10FCE000FE019E012B5F3F4F8FEF81932E173F0741
:10FCF000D8F76C877D87425F5F4F4C33510518F40E
:10FD00006CE370E001C0BA0182E2809300836093EB
:10FD10000A83E72FFF27E0930B831092088380E488
:10FD20008093098382E18093008320E030E02417F0
:10FD3000350750F4D7018D917D01809310832F5F9B
:10FD40003F4F24173507B0F39A014617570738F489
:10FD5000109210832F5F3F4F26173707C8F382E2B8
:10FD60008093008320E030E08091078386FD05C00A
:10FD70002F5F3F4F25313105B8F380E4809307832F
:10FD800060930583E09306838093048386E28093E7
:10FD900000838091008399279C012470307082FD3C
:10FDA000F8CFC901DF91CF911F910F91FF90EF9094
:10FDB0000895AF92BF92DF92EF92FF920F931F933D
:10FDC000CF93DF93CDB7DEB724970FB6F894DEBF9D
:10FDD0000FBECDBF5C017B0100E010E0DD24672B8E
:10FDE00009F4D6C021E0E114F104A1F0D09007831A
:10FDF0008D2D992782FF03C08FEF9FEFCAC080FD32
:10FE000009C0222319F40894E108F1082F5FE114D6
:10FE1000F10461F7D0FC03C0D0920783B9C082E639
:10FE2000809300839091078382E2809300834091C6
:10FE300003834F5F403608F04CE4491719F4D09221
:10FE400007839FC084E080930A8310920B831092F3
:10FE5000088340930983DE011196FD018AE08093B7
:10FE6000008320E030E08091108381932F5F3F4F2B
:10FE700024303105C0F382E28093008320E030E03B
:10FE80008091078386FD05C02F5F3F4F25313105E7
:10FE9000B8F380E48093078312962D913C911397D9
:10FEA000C90180549040835B954018F00E94B0FDDA
:10FEB00068C0898199278F709070019709F042C0BE
:10FEC00089010450104000930A83812F9927809361
:10FED0000B8384E080930883409309838AE08093B6
:10FEE0000083EEE0F1E0A80122E00335120710F0F4
:10FEF00042E552E020E030E02417350740F48091DD
:10FF0000108381932F5F3F4F24173507C0F32017CD
:10FF1000310738F4809110832F5F3F4F201731074E
:10FF2000C8F382E28093008320E030E08091078371
:10FF300086FD05C02F5F3F4F25313105B8F380E4C2
:10FF40008093078311968C911197815011968C9311
:10FF500011978C3420F48FE511968C93119711969C
:10FF60008C918093038380911A0190911B018A15D3
:10FF70009B0539F08850964011F40E944CFD00E03A
:10FF800010E0E114F10421F00115110509F42ACF64
:10FF9000C80124960FB6F894DEBF0FBECDBFDF9127
:10FFA000CF911F910F91FF90EF90DF90BF90AF9096
:10FFB00008952BE0660F771F881F991F2A95D1F7A8
:10FFC000161617061806190634F400006150704022
:10FFD00080409040D1F70895FC0103C0FC010B0163
:10FFE00061E060936800E8956091680060FDFCCF77
:04FFF000112408953B
:06FFF40000069800000069
:040000031000F000F9
:00000001FF
